:020000040000FA
:020000000528D1
:080008000529940195018316FE
:100010008B131F308500013086008111011481147B
:100020000115811283128501860101309100722031
:1000300006158617013091007220861306110611ED
:100040000130003C0319592886139020940086172C
:100050002030051E2E2805080F396220950014084F
:10006000543C031D412806150F30CE004E30CF0002
:10007000E33081008B178B160B11CB014B30AF2077
:1000800020281408523C031D4C2806118B128B1398
:10009000CB014B30AF2020281408433C031D5328CC
:1000A0001508AF2020281408493C031D5828592062
:1000B000202806158617013091007220FA20861339
:1000C0008613080082072034313432343334343418
:1000D0003534363437343834393430342A342334F0
:1000E00041344234FA308D008120FA308D00812075
:1000F000FA308D008120FA308D008120910B72281A
:1001000008008E308E00000000000000000000009B
:1001100000008E0B852800008D0B81280000080050
:100120000830960097014B180021061C9328A52043
:10013000061C93288617AA20970C97170618971362
:10014000960B9B28AA201708080043309300930BB6
:10015000A728080086309300930BAC28080099006C
:1001600009309800861400000000AA20980BBB28D4
:100170008610AA200800990C031CC0288610B528F8
:100180008614B5281008003C0130031CCF2800302D
:10019000031DCF280F08013C013003180301003C68
:1001A0000319E22810088C000F088F030F0A0319A7
:1001B00090031A089200E32006171A089200E32021
:1001C0000613C2280800920C920C3F3092050330AF
:1001D00092020000920BE92800000800FF309A000C
:1001E0008C01F0308F000C089000C22046308D004A
:1001F00081200800FF308D008120EE20EE200800D5
:100200008B128B130611CB010800CD000308CC0024
:10021000CF0B0D29CE03031912294C0883004D087A
:100220000B110900CB090B118B128B134C088300A7
:040230004D0809006C
:02400E00F13F80
:00000001FF
